 datadumpreq001

 Timestamp is 2eea2c8c (reproducible build file hash)

 Preferred load address is 0000000180000000

 Start         Length     Name                   Class
 0001:00000000 00003290H .text$mn                CODE
 0001:00003290 00000036H .text$mn$00             CODE
 0001:000032c6 00000092H .text$x                 CODE
 0002:00000000 000001c8H .idata$5                DATA
 0002:000001c8 00000038H .00cfg                  DATA
 0002:00000200 00000008H .CRT$XCA                DATA
 0002:00000208 00000008H .CRT$XCZ                DATA
 0002:00000210 00000008H .CRT$XIA                DATA
 0002:00000218 00000008H .CRT$XIC                DATA
 0002:00000220 00000008H .CRT$XIZ                DATA
 0002:00000228 00000008H .CRT$XLA                DATA
 0002:00000230 00000008H .CRT$XLZ                DATA
 0002:00000238 00000008H .CRT$XPA                DATA
 0002:00000240 00000008H .CRT$XPZ                DATA
 0002:00000248 00000008H .CRT$XTA                DATA
 0002:00000250 00000010H .CRT$XTZ                DATA
 0002:00000258 00000000H .gehcont$y              DATA
 0002:00000258 00000000H .gfids$y                DATA
 0002:00000260 00001f20H .rdata                  DATA
 0002:00002180 00000000H .rdata$CastGuardVftablesA DATA
 0002:00002180 00000000H .rdata$CastGuardVftablesC DATA
 0002:00002180 00000028H .rdata$T                DATA
 0002:000021a8 000000b8H .rdata$voltmd           DATA
 0002:00002260 00000320H .rdata$zzzdbg           DATA
 0002:00002580 00000008H .rtc$IAA                DATA
 0002:00002588 00000008H .rtc$IZZ                DATA
 0002:00002590 00000008H .rtc$TAA                DATA
 0002:00002598 00000008H .rtc$TZZ                DATA
 0002:000025a0 00000004H .tls                    DATA
 0002:000025a4 00000004H .tls$                   DATA
 0002:000025a8 00000008H .tls$ZZZ                DATA
 0002:000025b0 00000330H .xdata                  DATA
 0002:000028e0 000003acH .edata                  DATA
 0002:00002c8c 0000008cH .idata$2                DATA
 0002:00002d18 00000018H .idata$3                DATA
 0002:00002d30 000001c8H .idata$4                DATA
 0002:00002ef8 00000486H .idata$6                DATA
 0003:00000000 00000080H .data                   DATA
 0003:00000080 0001b378H .bss                    DATA
 0004:00000000 000003b4H .pdata                  DATA

  Address         Publics by Value              Rva+Base               Lib:Object

 0000:00000000       __AbsoluteZero             0000000000000000     <absolute>
 0000:00000000       ___safe_se_handler_count   0000000000000000     <absolute>
 0000:00000000       ___safe_se_handler_table   0000000000000000     <absolute>
 0000:00000000       __arm64x_extra_rfe_table   0000000000000000     <absolute>
 0000:00000000       __arm64x_extra_rfe_table_size 0000000000000000     <absolute>
 0000:00000000       __arm64x_native_entrypoint 0000000000000000     <absolute>
 0000:00000000       __arm64x_redirection_metadata 0000000000000000     <absolute>
 0000:00000000       __arm64x_redirection_metadata_count 0000000000000000     <absolute>
 0000:00000000       __dynamic_value_reloc_table 0000000000000000     <absolute>
 0000:00000000       __enclave_config           0000000000000000     <absolute>
 0000:00000000       __guard_check_icall_a64n_fptr 0000000000000000     <absolute>
 0000:00000000       __guard_eh_cont_count      0000000000000000     <absolute>
 0000:00000000       __guard_eh_cont_table      0000000000000000     <absolute>
 0000:00000000       __guard_fids_count         0000000000000000     <absolute>
 0000:00000000       __guard_fids_table         0000000000000000     <absolute>
 0000:00000000       __guard_iat_count          0000000000000000     <absolute>
 0000:00000000       __guard_iat_table          0000000000000000     <absolute>
 0000:00000000       __guard_longjmp_count      0000000000000000     <absolute>
 0000:00000000       __guard_longjmp_table      0000000000000000     <absolute>
 0000:00000000       __hybrid_auxiliary_iat     0000000000000000     <absolute>
 0000:00000000       __hybrid_auxiliary_iat_copy 0000000000000000     <absolute>
 0000:00000000       __hybrid_code_map          0000000000000000     <absolute>
 0000:00000000       __hybrid_code_map_count    0000000000000000     <absolute>
 0000:00000000       __x64_code_ranges_to_entry_points 0000000000000000     <absolute>
 0000:00000000       __x64_code_ranges_to_entry_points_count 0000000000000000     <absolute>
 0000:00000100       __guard_flags              0000000000000100     <absolute>
 0000:00000000       __ImageBase                0000000180000000     <linker-defined>
 0001:00000000       ?NewObject@JNIEnv_@@QEAAPEAV_jobject@@PEAV_jclass@@PEAU_jmethodID@@ZZ 0000000180001000 f i libdatadumpreq001.obj
 0001:00000024       ?SetEventNotificationMode@_jvmtiEnv@@QEAA?AW4jvmtiError@@W4jvmtiEventMode@@W4jvmtiEvent@@PEAV_jobject@@ZZ 0000000180001024 f i libdatadumpreq001.obj
 0001:0000002c       ?TranslateError@@YAPEBDW4jvmtiError@@@Z 000000018000102c f   libdatadumpreq001.obj
 0001:000002e4       ?TranslatePhase@@YAPEBDW4jvmtiPhase@@@Z 00000001800012e4 f   libdatadumpreq001.obj
 0001:00000330       ?nsk_jni_check_exception@@YAHPEAUJNIEnv_@@QEBDH@Z 0000000180001330 f   libdatadumpreq001.obj
 0001:00000474       ?nsk_jni_lverify@@YAHHPEAUJNIEnv_@@HQEBDH1ZZ 0000000180001474 f   libdatadumpreq001.obj
 0001:00000514       Agent_Initialize           0000000180001514 f   libdatadumpreq001.obj
 0001:0000074c       Agent_OnAttach             000000018000174c f   libdatadumpreq001.obj
 0001:0000074c       Agent_OnLoad               000000018000174c f   libdatadumpreq001.obj
 0001:00000858       Java_nsk_jvmti_DataDumpRequest_datadumpreq001_waitForResult 0000000180001858 f   libdatadumpreq001.obj
 0001:000008e0       Java_nsk_jvmti_unit_FollowReferences_FollowRefObjects_addRefToVerify 00000001800018e0 f   libdatadumpreq001.obj
 0001:00000a9c       Java_nsk_jvmti_unit_FollowReferences_FollowRefObjects_getTag 0000000180001a9c f   libdatadumpreq001.obj
 0001:00000b58       Java_nsk_jvmti_unit_FollowReferences_FollowRefObjects_resetRefsToVerify 0000000180001b58 f   libdatadumpreq001.obj
 0001:00000b60       Java_nsk_jvmti_unit_FollowReferences_FollowRefObjects_resetTags 0000000180001b60 f   libdatadumpreq001.obj
 0001:00000ba4       Java_nsk_jvmti_unit_FollowReferences_FollowRefObjects_setTag 0000000180001ba4 f   libdatadumpreq001.obj
 0001:00000df0       Java_nsk_share_jvmti_ArgumentHandler_getAgentOptionsString 0000000180001df0 f   libdatadumpreq001.obj
 0001:00000e9c       Java_nsk_share_jvmti_DebugeeClass_checkStatus 0000000180001e9c f   libdatadumpreq001.obj
 0001:00000f24       Java_nsk_share_jvmti_DebugeeClass_resetAgentData 0000000180001f24 f   libdatadumpreq001.obj
 0001:00000f84       Java_nsk_share_jvmti_RedefineAgent_agentStatus 0000000180001f84 f   libdatadumpreq001.obj
 0001:00000f90       Java_nsk_share_jvmti_RedefineAgent_isRedefined 0000000180001f90 f   libdatadumpreq001.obj
 0001:00000f9c       Java_nsk_share_jvmti_RedefineAgent_redefineAttempted 0000000180001f9c f   libdatadumpreq001.obj
 0001:00000fa8       MA_checkStatus             0000000180001fa8 f   libdatadumpreq001.obj
 0001:0000104c       __local_stdio_printf_options 000000018000204c f i libdatadumpreq001.obj
 0001:000013e0       createRawMonitor           00000001800023e0 f   libdatadumpreq001.obj
 0001:00001468       exitOnError                0000000180002468 f   libdatadumpreq001.obj
 0001:0000151c       fprintf                    000000018000251c f i libdatadumpreq001.obj
 0001:00001560       nsk_complain               0000000180002560 f   libdatadumpreq001.obj
 0001:0000158c       nsk_jvmti_createJVMTIEnv   000000018000258c f   libdatadumpreq001.obj
 0001:000016bc       nsk_jvmti_lverify          00000001800026bc f   libdatadumpreq001.obj
 0001:000017ac       nsk_jvmti_parseOptions     00000001800027ac f   libdatadumpreq001.obj
 0001:000019fc       nsk_jvmti_resetAgentData   00000001800029fc f   libdatadumpreq001.obj
 0001:00001a70       nsk_lcomplain              0000000180002a70 f   libdatadumpreq001.obj
 0001:00001a90       nsk_ldisplay               0000000180002a90 f   libdatadumpreq001.obj
 0001:00001ab0       nsk_ltrace                 0000000180002ab0 f   libdatadumpreq001.obj
 0001:00001ad0       nsk_lvcomplain             0000000180002ad0 f   libdatadumpreq001.obj
 0001:00001c88       nsk_lvdisplay              0000000180002c88 f   libdatadumpreq001.obj
 0001:00001cd4       nsk_lverify                0000000180002cd4 f   libdatadumpreq001.obj
 0001:00001d30       nsk_lvtrace                0000000180002d30 f   libdatadumpreq001.obj
 0001:00001d90       nsk_printf                 0000000180002d90 f   libdatadumpreq001.obj
 0001:00001db8       nsk_vprintf                0000000180002db8 f   libdatadumpreq001.obj
 0001:00001e6c       printf                     0000000180002e6c f i libdatadumpreq001.obj
 0001:0000236c       __raise_securityfailure    000000018000336c f   MSVCRT:gs_report.obj
 0001:000023a0       __report_gsfailure         00000001800033a0 f   MSVCRT:gs_report.obj
 0001:000025e0       __GSHandlerCheck           00000001800035e0 f   MSVCRT:gshandler.obj
 0001:00002600       __GSHandlerCheckCommon     0000000180003600 f   MSVCRT:gshandler.obj
 0001:00002670       __security_check_cookie    0000000180003670 f   MSVCRT:amdsecgs.obj
 0001:000029b0       _DllMainCRTStartup         00000001800039b0 f   MSVCRT:dll_dllmain.obj
 0001:000029f0       __scrt_acquire_startup_lock 00000001800039f0 f   MSVCRT:utility.obj
 0001:00002a2c       __scrt_dllmain_after_initialize_c 0000000180003a2c f   MSVCRT:utility.obj
 0001:00002a60       __scrt_dllmain_before_initialize_c 0000000180003a60 f   MSVCRT:utility.obj
 0001:00002a78       __scrt_dllmain_crt_thread_attach 0000000180003a78 f   MSVCRT:utility.obj
 0001:00002aa0       __scrt_dllmain_crt_thread_detach 0000000180003aa0 f   MSVCRT:utility.obj
 0001:00002ab8       __scrt_dllmain_exception_filter 0000000180003ab8 f   MSVCRT:utility.obj
 0001:00002b18       __scrt_dllmain_uninitialize_c 0000000180003b18 f   MSVCRT:utility.obj
 0001:00002b48       __scrt_dllmain_uninitialize_critical 0000000180003b48 f   MSVCRT:utility.obj
 0001:00002b5c       __scrt_initialize_crt      0000000180003b5c f   MSVCRT:utility.obj
 0001:00002ba8       __scrt_initialize_onexit_tables 0000000180003ba8 f   MSVCRT:utility.obj
 0001:00002c34       __scrt_is_nonwritable_in_current_image 0000000180003c34 f   MSVCRT:utility.obj
 0001:00002ccc       __scrt_release_startup_lock 0000000180003ccc f   MSVCRT:utility.obj
 0001:00002cf0       __scrt_uninitialize_crt    0000000180003cf0 f   MSVCRT:utility.obj
 0001:00002d1c       _onexit                    0000000180003d1c f   MSVCRT:utility.obj
 0001:00002d58       atexit                     0000000180003d58 f   MSVCRT:utility.obj
 0001:00002d70       __crt_debugger_hook        0000000180003d70 f   MSVCRT:utility_desktop.obj
 0001:00002d78       __scrt_fastfail            0000000180003d78 f   MSVCRT:utility_desktop.obj
 0001:00002ec4       _guard_check_icall_nop     0000000180003ec4 f i MSVCRT:guard_support.obj
 0001:00002ec8       __security_init_cookie     0000000180003ec8 f   MSVCRT:gs_support.obj
 0001:00002f74       DllMain                    0000000180003f74 f   MSVCRT:dll_dllmain_stub.obj
 0001:00002f98       ?__scrt_initialize_type_info@@YAXXZ 0000000180003f98 f   MSVCRT:tncleanup.obj
 0001:00002fa8       ?__scrt_uninitialize_type_info@@YAXXZ 0000000180003fa8 f   MSVCRT:tncleanup.obj
 0001:00002fb4       __local_stdio_scanf_options 0000000180003fb4 f i MSVCRT:default_local_stdio_options.obj
 0001:00002fbc       __scrt_initialize_default_local_stdio_options 0000000180003fbc f   MSVCRT:default_local_stdio_options.obj
 0001:00002fd8       __scrt_get_dyn_tls_init_callback 0000000180003fd8 f   MSVCRT:dyn_tls_init.obj
 0001:00002fe0       _RTC_Initialize            0000000180003fe0 f   MSVCRT:initsect.obj
 0001:0000301c       _RTC_Terminate             000000018000401c f   MSVCRT:initsect.obj
 0001:00003058       __isa_available_init       0000000180004058 f   MSVCRT:cpu_disp.obj
 0001:00003204       _get_startup_argv_mode     0000000180004204 f   MSVCRT:argv_mode.obj
 0001:0000320c       __scrt_is_ucrt_dll_in_use  000000018000420c f   MSVCRT:ucrt_detection.obj
 0001:00003220       memcpy                     0000000180004220 f   vcruntime:VCRUNTIME140.dll
 0001:00003226       memset                     0000000180004226 f   vcruntime:VCRUNTIME140.dll
 0001:0000322c       strchr                     000000018000422c f   vcruntime:VCRUNTIME140.dll
 0001:00003232       __C_specific_handler       0000000180004232 f   vcruntime:VCRUNTIME140.dll
 0001:00003238       __std_type_info_destroy_list 0000000180004238 f   vcruntime:VCRUNTIME140.dll
 0001:0000323e       strcmp                     000000018000423e f   ucrt:api-ms-win-crt-string-l1-1-0.dll
 0001:00003244       strlen                     0000000180004244 f   ucrt:api-ms-win-crt-string-l1-1-0.dll
 0001:0000324a       _initterm                  000000018000424a f   ucrt:api-ms-win-crt-runtime-l1-1-0.dll
 0001:00003250       _initterm_e                0000000180004250 f   ucrt:api-ms-win-crt-runtime-l1-1-0.dll
 0001:00003256       _seh_filter_dll            0000000180004256 f   ucrt:api-ms-win-crt-runtime-l1-1-0.dll
 0001:0000325c       _configure_narrow_argv     000000018000425c f   ucrt:api-ms-win-crt-runtime-l1-1-0.dll
 0001:00003262       _initialize_narrow_environment 0000000180004262 f   ucrt:api-ms-win-crt-runtime-l1-1-0.dll
 0001:00003268       _initialize_onexit_table   0000000180004268 f   ucrt:api-ms-win-crt-runtime-l1-1-0.dll
 0001:0000326e       _register_onexit_function  000000018000426e f   ucrt:api-ms-win-crt-runtime-l1-1-0.dll
 0001:00003274       _execute_onexit_table      0000000180004274 f   ucrt:api-ms-win-crt-runtime-l1-1-0.dll
 0001:0000327a       _crt_atexit                000000018000427a f   ucrt:api-ms-win-crt-runtime-l1-1-0.dll
 0001:00003280       _cexit                     0000000180004280 f   ucrt:api-ms-win-crt-runtime-l1-1-0.dll
 0001:00003288       __acrt_initialize          0000000180004288 f   MSVCRT:ucrt_stubs.obj
 0001:00003288       __acrt_thread_attach       0000000180004288 f   MSVCRT:ucrt_stubs.obj
 0001:00003288       __acrt_thread_detach       0000000180004288 f   MSVCRT:ucrt_stubs.obj
 0001:00003288       __acrt_uninitialize        0000000180004288 f   MSVCRT:ucrt_stubs.obj
 0001:00003288       __acrt_uninitialize_critical 0000000180004288 f   MSVCRT:ucrt_stubs.obj
 0001:00003288       __scrt_stub_for_acrt_initialize 0000000180004288 f   MSVCRT:ucrt_stubs.obj
 0001:00003288       __scrt_stub_for_acrt_thread_attach 0000000180004288 f   MSVCRT:ucrt_stubs.obj
 0001:00003288       __scrt_stub_for_acrt_thread_detach 0000000180004288 f   MSVCRT:ucrt_stubs.obj
 0001:00003288       __scrt_stub_for_acrt_uninitialize 0000000180004288 f   MSVCRT:ucrt_stubs.obj
 0001:00003288       __scrt_stub_for_acrt_uninitialize_critical 0000000180004288 f   MSVCRT:ucrt_stubs.obj
 0001:00003288       __vcrt_initialize          0000000180004288 f   MSVCRT:ucrt_stubs.obj
 0001:00003288       __vcrt_thread_attach       0000000180004288 f   MSVCRT:ucrt_stubs.obj
 0001:00003288       __vcrt_thread_detach       0000000180004288 f   MSVCRT:ucrt_stubs.obj
 0001:00003288       __vcrt_uninitialize        0000000180004288 f   MSVCRT:ucrt_stubs.obj
 0001:00003288       __vcrt_uninitialize_critical 0000000180004288 f   MSVCRT:ucrt_stubs.obj
 0001:0000328c       __scrt_stub_for_is_c_termination_complete 000000018000428c f   MSVCRT:ucrt_stubs.obj
 0001:0000328c       _is_c_termination_complete 000000018000428c f   MSVCRT:ucrt_stubs.obj
 0001:000032a0       _guard_dispatch_icall_nop  00000001800042a0 f   MSVCRT:guard_dispatch.obj
 0001:000032c0       _guard_xfg_dispatch_icall_nop 00000001800042c0 f   MSVCRT:guard_xfg_dispatch.obj
 0002:00000000       __imp_RtlCaptureContext    0000000180005000     kernel32:KERNEL32.dll
 0002:00000008       __imp_RtlLookupFunctionEntry 0000000180005008     kernel32:KERNEL32.dll
 0002:00000010       __imp_RtlVirtualUnwind     0000000180005010     kernel32:KERNEL32.dll
 0002:00000018       __imp_UnhandledExceptionFilter 0000000180005018     kernel32:KERNEL32.dll
 0002:00000020       __imp_SetUnhandledExceptionFilter 0000000180005020     kernel32:KERNEL32.dll
 0002:00000028       __imp_GetCurrentProcess    0000000180005028     kernel32:KERNEL32.dll
 0002:00000030       __imp_TerminateProcess     0000000180005030     kernel32:KERNEL32.dll
 0002:00000038       __imp_IsProcessorFeaturePresent 0000000180005038     kernel32:KERNEL32.dll
 0002:00000040       __imp_CloseHandle          0000000180005040     kernel32:KERNEL32.dll
 0002:00000048       __imp_InitializeCriticalSectionAndSpinCount 0000000180005048     kernel32:KERNEL32.dll
 0002:00000050       __imp_DeleteCriticalSection 0000000180005050     kernel32:KERNEL32.dll
 0002:00000058       __imp_CreateEventW         0000000180005058     kernel32:KERNEL32.dll
 0002:00000060       __imp_GetModuleHandleW     0000000180005060     kernel32:KERNEL32.dll
 0002:00000068       __imp_GetProcAddress       0000000180005068     kernel32:KERNEL32.dll
 0002:00000070       __imp_IsDebuggerPresent    0000000180005070     kernel32:KERNEL32.dll
 0002:00000078       __imp_QueryPerformanceCounter 0000000180005078     kernel32:KERNEL32.dll
 0002:00000080       __imp_GetCurrentProcessId  0000000180005080     kernel32:KERNEL32.dll
 0002:00000088       __imp_GetCurrentThreadId   0000000180005088     kernel32:KERNEL32.dll
 0002:00000090       __imp_GetSystemTimeAsFileTime 0000000180005090     kernel32:KERNEL32.dll
 0002:00000098       __imp_DisableThreadLibraryCalls 0000000180005098     kernel32:KERNEL32.dll
 0002:000000a0       __imp_InitializeSListHead  00000001800050a0     kernel32:KERNEL32.dll
 0002:000000a8       \177KERNEL32_NULL_THUNK_DATA 00000001800050a8     kernel32:KERNEL32.dll
 0002:000000b0       __imp_memcpy               00000001800050b0     vcruntime:VCRUNTIME140.dll
 0002:000000b8       __imp_memset               00000001800050b8     vcruntime:VCRUNTIME140.dll
 0002:000000c0       __imp_strchr               00000001800050c0     vcruntime:VCRUNTIME140.dll
 0002:000000c8       __imp___C_specific_handler 00000001800050c8     vcruntime:VCRUNTIME140.dll
 0002:000000d0       __imp___std_type_info_destroy_list 00000001800050d0     vcruntime:VCRUNTIME140.dll
 0002:000000d8       \177VCRUNTIME140_NULL_THUNK_DATA 00000001800050d8     vcruntime:VCRUNTIME140.dll
 0002:000000e0       __imp_strtol               00000001800050e0     ucrt:api-ms-win-crt-convert-l1-1-0.dll
 0002:000000e8       \177api-ms-win-crt-convert-l1-1-0_NULL_THUNK_DATA 00000001800050e8     ucrt:api-ms-win-crt-convert-l1-1-0.dll
 0002:000000f0       __imp_malloc               00000001800050f0     ucrt:api-ms-win-crt-heap-l1-1-0.dll
 0002:000000f8       __imp_free                 00000001800050f8     ucrt:api-ms-win-crt-heap-l1-1-0.dll
 0002:00000100       \177api-ms-win-crt-heap-l1-1-0_NULL_THUNK_DATA 0000000180005100     ucrt:api-ms-win-crt-heap-l1-1-0.dll
 0002:00000108       __imp__errno               0000000180005108     ucrt:api-ms-win-crt-runtime-l1-1-0.dll
 0002:00000110       __imp_exit                 0000000180005110     ucrt:api-ms-win-crt-runtime-l1-1-0.dll
 0002:00000118       __imp__cexit               0000000180005118     ucrt:api-ms-win-crt-runtime-l1-1-0.dll
 0002:00000120       __imp__crt_atexit          0000000180005120     ucrt:api-ms-win-crt-runtime-l1-1-0.dll
 0002:00000128       __imp__execute_onexit_table 0000000180005128     ucrt:api-ms-win-crt-runtime-l1-1-0.dll
 0002:00000130       __imp__register_onexit_function 0000000180005130     ucrt:api-ms-win-crt-runtime-l1-1-0.dll
 0002:00000138       __imp__initialize_onexit_table 0000000180005138     ucrt:api-ms-win-crt-runtime-l1-1-0.dll
 0002:00000140       __imp__initialize_narrow_environment 0000000180005140     ucrt:api-ms-win-crt-runtime-l1-1-0.dll
 0002:00000148       __imp__configure_narrow_argv 0000000180005148     ucrt:api-ms-win-crt-runtime-l1-1-0.dll
 0002:00000150       __imp__seh_filter_dll      0000000180005150     ucrt:api-ms-win-crt-runtime-l1-1-0.dll
 0002:00000158       __imp__initterm_e          0000000180005158     ucrt:api-ms-win-crt-runtime-l1-1-0.dll
 0002:00000160       __imp__initterm            0000000180005160     ucrt:api-ms-win-crt-runtime-l1-1-0.dll
 0002:00000168       \177api-ms-win-crt-runtime-l1-1-0_NULL_THUNK_DATA 0000000180005168     ucrt:api-ms-win-crt-runtime-l1-1-0.dll
 0002:00000170       __imp___acrt_iob_func      0000000180005170     ucrt:api-ms-win-crt-stdio-l1-1-0.dll
 0002:00000178       __imp_fflush               0000000180005178     ucrt:api-ms-win-crt-stdio-l1-1-0.dll
 0002:00000180       __imp___stdio_common_vsprintf 0000000180005180     ucrt:api-ms-win-crt-stdio-l1-1-0.dll
 0002:00000188       __imp___stdio_common_vfprintf 0000000180005188     ucrt:api-ms-win-crt-stdio-l1-1-0.dll
 0002:00000190       \177api-ms-win-crt-stdio-l1-1-0_NULL_THUNK_DATA 0000000180005190     ucrt:api-ms-win-crt-stdio-l1-1-0.dll
 0002:00000198       __imp_strcmp               0000000180005198     ucrt:api-ms-win-crt-string-l1-1-0.dll
 0002:000001a0       __imp__strdup              00000001800051a0     ucrt:api-ms-win-crt-string-l1-1-0.dll
 0002:000001a0       __imp_strdup               00000001800051a0     ucrt:api-ms-win-crt-string-l1-1-0.dll
 0002:000001a8       __imp_strlen               00000001800051a8     ucrt:api-ms-win-crt-string-l1-1-0.dll
 0002:000001b0       __imp_strpbrk              00000001800051b0     ucrt:api-ms-win-crt-string-l1-1-0.dll
 0002:000001b8       __imp_strncpy              00000001800051b8     ucrt:api-ms-win-crt-string-l1-1-0.dll
 0002:000001c0       \177api-ms-win-crt-string-l1-1-0_NULL_THUNK_DATA 00000001800051c0     ucrt:api-ms-win-crt-string-l1-1-0.dll
 0002:000001c8       __guard_check_icall_fptr   00000001800051c8     MSVCRT:guard_support.obj
 0002:000001d0       __guard_xfg_check_icall_fptr 00000001800051d0     MSVCRT:guard_support.obj
 0002:000001d8       __guard_dispatch_icall_fptr 00000001800051d8     MSVCRT:guard_support.obj
 0002:000001e0       __guard_xfg_dispatch_icall_fptr 00000001800051e0     MSVCRT:guard_support.obj
 0002:000001e8       __guard_xfg_table_dispatch_icall_fptr 00000001800051e8     MSVCRT:guard_support.obj
 0002:000001f0       __castguard_check_failure_os_handled_fptr 00000001800051f0     MSVCRT:guard_support.obj
 0002:000001f8       __guard_memcpy_fptr        00000001800051f8     vcruntime:softmemtag.obj
 0002:00000200       __xc_a                     0000000180005200     MSVCRT:initializers.obj
 0002:00000208       __xc_z                     0000000180005208     MSVCRT:initializers.obj
 0002:00000210       __xi_a                     0000000180005210     MSVCRT:initializers.obj
 0002:00000220       __xi_z                     0000000180005220     MSVCRT:initializers.obj
 0002:00000228       __xl_a                     0000000180005228     MSVCRT:tlssup.obj
 0002:00000230       __xl_z                     0000000180005230     MSVCRT:tlssup.obj
 0002:00000238       __xp_a                     0000000180005238     MSVCRT:initializers.obj
 0002:00000240       __xp_z                     0000000180005240     MSVCRT:initializers.obj
 0002:00000248       __xt_a                     0000000180005248     MSVCRT:initializers.obj
 0002:00000250       __xt_z                     0000000180005250     MSVCRT:initializers.obj
 0002:00000260       g_refKindStr               0000000180005260     libdatadumpreq001.obj
 0002:00000410       ??_C@_09BPLDFGCI@unknown_0@ 0000000180005410     libdatadumpreq001.obj
 0002:00000420       ??_C@_0BL@FPNMECJD@JVMTI_HEAP_REFERENCE_CLASS@ 0000000180005420     libdatadumpreq001.obj
 0002:00000440       ??_C@_0BL@FKGKKLNM@JVMTI_HEAP_REFERENCE_FIELD@ 0000000180005440     libdatadumpreq001.obj
 0002:00000460       ??_C@_0CD@CAEHCFJF@JVMTI_HEAP_REFERENCE_ARRAY_ELEM@ 0000000180005460     libdatadumpreq001.obj
 0002:00000488       ??_C@_0CC@DNEBMCNK@JVMTI_HEAP_REFERENCE_CLASS_LOAD@ 0000000180005488     libdatadumpreq001.obj
 0002:000004b0       ??_C@_0BN@CJMIPEBB@JVMTI_HEAP_REFERENCE_SIGNERS@ 00000001800054b0     libdatadumpreq001.obj
 0002:000004d0       ??_C@_0CH@HBOIDPEB@JVMTI_HEAP_REFERENCE_PROTECTION@ 00000001800054d0     libdatadumpreq001.obj
 0002:000004f8       ??_C@_0BP@MDKGDGKL@JVMTI_HEAP_REFERENCE_INTERFACE@ 00000001800054f8     libdatadumpreq001.obj
 0002:00000518       ??_C@_0CC@JJMIHNJH@JVMTI_HEAP_REFERENCE_STATIC_FIE@ 0000000180005518     libdatadumpreq001.obj
 0002:00000540       ??_C@_0CD@IDHEEGID@JVMTI_HEAP_REFERENCE_CONSTANT_P@ 0000000180005540     libdatadumpreq001.obj
 0002:00000568       ??_C@_0CA@EFFCHNG@JVMTI_HEAP_REFERENCE_SUPERCLASS@ 0000000180005568     libdatadumpreq001.obj
 0002:00000588       ??_C@_0L@PCDFHGCJ@unknown_11@ 0000000180005588     libdatadumpreq001.obj
 0002:00000598       ??_C@_0L@NJBICFOK@unknown_12@ 0000000180005598     libdatadumpreq001.obj
 0002:000005a8       ??_C@_0L@MAADBEKL@unknown_13@ 00000001800055a8     libdatadumpreq001.obj
 0002:000005b8       ??_C@_0L@IPECICGM@unknown_14@ 00000001800055b8     libdatadumpreq001.obj
 0002:000005c8       ??_C@_0L@JGFJLDCN@unknown_15@ 00000001800055c8     libdatadumpreq001.obj
 0002:000005d8       ??_C@_0L@LNHEOAOO@unknown_16@ 00000001800055d8     libdatadumpreq001.obj
 0002:000005e8       ??_C@_0L@KEGPNBKP@unknown_17@ 00000001800055e8     libdatadumpreq001.obj
 0002:000005f8       ??_C@_0L@CDPHMNGA@unknown_18@ 00000001800055f8     libdatadumpreq001.obj
 0002:00000608       ??_C@_0L@DKOMPMCB@unknown_19@ 0000000180005608     libdatadumpreq001.obj
 0002:00000618       ??_C@_0L@OJGIPJDB@unknown_20@ 0000000180005618     libdatadumpreq001.obj
 0002:00000628       ??_C@_0CA@KAOFNDEM@JVMTI_HEAP_REFERENCE_JNI_GLOBAL@ 0000000180005628     libdatadumpreq001.obj
 0002:00000648       ??_C@_0CC@HPFAJBK@JVMTI_HEAP_REFERENCE_SYSTEM_CLA@ 0000000180005648     libdatadumpreq001.obj
 0002:00000670       ??_C@_0BN@FDEGFOHC@JVMTI_HEAP_REFERENCE_MONITOR@ 0000000180005670     libdatadumpreq001.obj
 0002:00000690       ??_C@_0CB@HKIBCMAJ@JVMTI_HEAP_REFERENCE_STACK_LOCA@ 0000000180005690     libdatadumpreq001.obj
 0002:000006b8       ??_C@_0BP@EAACMMOE@JVMTI_HEAP_REFERENCE_JNI_LOCAL@ 00000001800056b8     libdatadumpreq001.obj
 0002:000006d8       ??_C@_0BM@IJDEOGOE@JVMTI_HEAP_REFERENCE_THREAD@ 00000001800056d8     libdatadumpreq001.obj
 0002:000006f8       ??_C@_0BL@EDGPPKC@JVMTI_HEAP_REFERENCE_OTHER@ 00000001800056f8     libdatadumpreq001.obj
 0002:00000714       ??_C@_04BCJPDBDA@Code@     0000000180005714     libdatadumpreq001.obj
 0002:00000720       ??_C@_0BA@OCLMCFKC@LineNumberTable@ 0000000180005720     libdatadumpreq001.obj
 0002:00000730       ??_C@_0BD@CPAEPILC@LocalVariableTable@ 0000000180005730     libdatadumpreq001.obj
 0002:00000748       ??_C@_0BH@NMBDNHBD@LocalVariableTypeTable@ 0000000180005748     libdatadumpreq001.obj
 0002:00000760       ??_C@_0O@HIHEEDNJ@StackMapTable@ 0000000180005760     libdatadumpreq001.obj
 0002:00000770       ??_C@_0L@HCDIAMJG@?9?5?$CFs?0?5?$CFd?3?5@ 0000000180005770     libdatadumpreq001.obj
 0002:00000780       ??_C@_0JI@HLPECLFI@?$CD?5?4?4?4?6?$CD?5ERROR?3?5too?5many?5complai@ 0000000180005780     libdatadumpreq001.obj
 0002:00000820       ??_C@_0ED@JNEKCCOB@The?5following?5fake?5exception?5st@ 0000000180005820     libdatadumpreq001.obj
 0002:00000868       ??_C@_0CN@FCNMDFBH@nsk?4share?4Fake_Exception_for_RU@ 0000000180005868     libdatadumpreq001.obj
 0002:00000898       ??_C@_08PGFFNAEI@?$CI?$CFs?3?$CFd?$CJ?5@ 0000000180005898     libdatadumpreq001.obj
 0002:000008a8       ??_C@_0DP@IENMAEGI@s?2test?2hotspot?2jtreg?2vmTestbase@ 00000001800058a8     libdatadumpreq001.obj
 0002:000008e8       ??_C@_0BL@NDJLFFJB@?7at?5nsk_lvcomplain?$CI?$CFs?3?$CFd?$CJ?6@ 00000001800058e8     libdatadumpreq001.obj
 0002:00000908       ??_C@_0BC@JOOKAFKF@?$CD?5ERROR?3?5?$CFs?0?5?$CFd?3?5@ 0000000180005908     libdatadumpreq001.obj
 0002:00000920       ??_C@_09KJEAHMEH@?$CD?5ERROR?3?5@ 0000000180005920     libdatadumpreq001.obj
 0002:0000092c       ??_C@_02GPIOPFAK@?$DO?$DO@ 000000018000592c     libdatadumpreq001.obj
 0002:00000930       ??_C@_02FODMEDOG@?$DM?$DM@ 0000000180005930     libdatadumpreq001.obj
 0002:00000934       ??_C@_02DJGKEECL@?4?4@     0000000180005934     libdatadumpreq001.obj
 0002:00000938       ??_C@_0O@CJPGJOAF@?9?5?$CFs?0?5?$CFd?3?5?$CFs?5@ 0000000180005938     libdatadumpreq001.obj
 0002:00000948       ??_C@_0CB@IAKPDOIC@?$CD?5?5?5verified?5assertion?5is?5FALSE@ 0000000180005948     libdatadumpreq001.obj
 0002:00000970       ??_C@_0CO@LGONDEPD@stdout?3?5fflush?5failed?5?9?5err?$DN?$CFd?5@ 0000000180005970     libdatadumpreq001.obj
 0002:000009a0       ??_C@_0CO@KBGKJPBD@stderr?3?5fflush?5failed?5?9?5err?$DN?$CFd?5@ 00000001800059a0     libdatadumpreq001.obj
 0002:000009d0       ??_C@_0BB@JCNMKLLK@JVMTI_ERROR_NONE@ 00000001800059d0     libdatadumpreq001.obj
 0002:000009e8       ??_C@_0BL@LDIMKLPH@JVMTI_ERROR_INVALID_THREAD@ 00000001800059e8     libdatadumpreq001.obj
 0002:00000a08       ??_C@_0CB@PJFPAIKJ@JVMTI_ERROR_INVALID_THREAD_GROU@ 0000000180005a08     libdatadumpreq001.obj
 0002:00000a30       ??_C@_0BN@LLMKHMNF@JVMTI_ERROR_INVALID_PRIORITY@ 0000000180005a30     libdatadumpreq001.obj
 0002:00000a50       ??_C@_0CB@MBOFKAGB@JVMTI_ERROR_THREAD_NOT_SUSPENDE@ 0000000180005a50     libdatadumpreq001.obj
 0002:00000a78       ??_C@_0BN@FABOLPBI@JVMTI_ERROR_THREAD_SUSPENDED@ 0000000180005a78     libdatadumpreq001.obj
 0002:00000a98       ??_C@_0BN@FDGNOBJM@JVMTI_ERROR_THREAD_NOT_ALIVE@ 0000000180005a98     libdatadumpreq001.obj
 0002:00000ab8       ??_C@_0BL@GOBIFKNJ@JVMTI_ERROR_INVALID_OBJECT@ 0000000180005ab8     libdatadumpreq001.obj
 0002:00000ad8       ??_C@_0BK@FCMAJPPC@JVMTI_ERROR_INVALID_CLASS@ 0000000180005ad8     libdatadumpreq001.obj
 0002:00000af8       ??_C@_0BP@IKLLBKEB@JVMTI_ERROR_CLASS_NOT_PREPARED@ 0000000180005af8     libdatadumpreq001.obj
 0002:00000b18       ??_C@_0BN@KLPPLKG@JVMTI_ERROR_INVALID_METHODID@ 0000000180005b18     libdatadumpreq001.obj
 0002:00000b38       ??_C@_0BN@BCEKOKND@JVMTI_ERROR_INVALID_LOCATION@ 0000000180005b38     libdatadumpreq001.obj
 0002:00000b58       ??_C@_0BM@DFDGPME@JVMTI_ERROR_INVALID_FIELDID@ 0000000180005b58     libdatadumpreq001.obj
 0002:00000b78       ??_C@_0BL@NELIEPEC@JVMTI_ERROR_NO_MORE_FRAMES@ 0000000180005b78     libdatadumpreq001.obj
 0002:00000b98       ??_C@_0BJ@BDBECFDM@JVMTI_ERROR_OPAQUE_FRAME@ 0000000180005b98     libdatadumpreq001.obj
 0002:00000bb8       ??_C@_0BK@MIIFNLOB@JVMTI_ERROR_TYPE_MISMATCH@ 0000000180005bb8     libdatadumpreq001.obj
 0002:00000bd8       ??_C@_0BJ@HPCAOILC@JVMTI_ERROR_INVALID_SLOT@ 0000000180005bd8     libdatadumpreq001.obj
 0002:00000bf8       ??_C@_0BG@CHILOPNI@JVMTI_ERROR_DUPLICATE@ 0000000180005bf8     libdatadumpreq001.obj
 0002:00000c10       ??_C@_0BG@DIEMLHKM@JVMTI_ERROR_NOT_FOUND@ 0000000180005c10     libdatadumpreq001.obj
 0002:00000c28       ??_C@_0BM@NHMCKHOB@JVMTI_ERROR_INVALID_MONITOR@ 0000000180005c28     libdatadumpreq001.obj
 0002:00000c48       ??_C@_0BO@PPEDAJGL@JVMTI_ERROR_NOT_MONITOR_OWNER@ 0000000180005c48     libdatadumpreq001.obj
 0002:00000c68       ??_C@_0BG@FCAIPEID@JVMTI_ERROR_INTERRUPT@ 0000000180005c68     libdatadumpreq001.obj
 0002:00000c80       ??_C@_0CB@EGDBNKOI@JVMTI_ERROR_INVALID_CLASS_FORMA@ 0000000180005c80     libdatadumpreq001.obj
 0002:00000ca8       ??_C@_0CG@DGKOGIAL@JVMTI_ERROR_CIRCULAR_CLASS_DEFI@ 0000000180005ca8     libdatadumpreq001.obj
 0002:00000cd0       ??_C@_0BP@ICEALPKC@JVMTI_ERROR_FAILS_VERIFICATION@ 0000000180005cd0     libdatadumpreq001.obj
 0002:00000cf0       ??_C@_0DC@JDACLMIO@JVMTI_ERROR_UNSUPPORTED_REDEFIN@ 0000000180005cf0     libdatadumpreq001.obj
 0002:00000d28       ??_C@_0DE@GKDKNOMJ@JVMTI_ERROR_UNSUPPORTED_REDEFIN@ 0000000180005d28     libdatadumpreq001.obj
 0002:00000d60       ??_C@_0BO@LAFKIOG@JVMTI_ERROR_INVALID_TYPESTATE@ 0000000180005d60     libdatadumpreq001.obj
 0002:00000d80       ??_C@_0DH@INDGCLLB@JVMTI_ERROR_UNSUPPORTED_REDEFIN@ 0000000180005d80     libdatadumpreq001.obj
 0002:00000db8       ??_C@_0DE@NHEOMMGI@JVMTI_ERROR_UNSUPPORTED_REDEFIN@ 0000000180005db8     libdatadumpreq001.obj
 0002:00000df0       ??_C@_0CA@EKPNJOEP@JVMTI_ERROR_UNSUPPORTED_VERSION@ 0000000180005df0     libdatadumpreq001.obj
 0002:00000e10       ??_C@_0BN@OFFMAHHL@JVMTI_ERROR_NAMES_DONT_MATCH@ 0000000180005e10     libdatadumpreq001.obj
 0002:00000e30       ??_C@_0DN@HHBBLAKE@JVMTI_ERROR_UNSUPPORTED_REDEFIN@ 0000000180005e30     libdatadumpreq001.obj
 0002:00000e70       ??_C@_0DO@HMBGBGNA@JVMTI_ERROR_UNSUPPORTED_REDEFIN@ 0000000180005e70     libdatadumpreq001.obj
 0002:00000eb0       ??_C@_0BP@PBECGKHJ@JVMTI_ERROR_UNMODIFIABLE_CLASS@ 0000000180005eb0     libdatadumpreq001.obj
 0002:00000ed0       ??_C@_0BK@CANILEHF@JVMTI_ERROR_NOT_AVAILABLE@ 0000000180005ed0     libdatadumpreq001.obj
 0002:00000ef0       ??_C@_0CE@INJKMEFK@JVMTI_ERROR_MUST_POSSESS_CAPABI@ 0000000180005ef0     libdatadumpreq001.obj
 0002:00000f18       ??_C@_0BJ@LBFPFPDM@JVMTI_ERROR_NULL_POINTER@ 0000000180005f18     libdatadumpreq001.obj
 0002:00000f38       ??_C@_0BP@CHJPNNEM@JVMTI_ERROR_ABSENT_INFORMATION@ 0000000180005f38     libdatadumpreq001.obj
 0002:00000f58       ??_C@_0BP@OMFMNLC@JVMTI_ERROR_INVALID_EVENT_TYPE@ 0000000180005f58     libdatadumpreq001.obj
 0002:00000f78       ??_C@_0BN@BIBNPHHO@JVMTI_ERROR_ILLEGAL_ARGUMENT@ 0000000180005f78     libdatadumpreq001.obj
 0002:00000f98       ??_C@_0BK@KKNDHDCE@JVMTI_ERROR_NATIVE_METHOD@ 0000000180005f98     libdatadumpreq001.obj
 0002:00000fb8       ??_C@_0BK@PMKCFHAE@JVMTI_ERROR_OUT_OF_MEMORY@ 0000000180005fb8     libdatadumpreq001.obj
 0002:00000fd8       ??_C@_0BK@NNJBDMNB@JVMTI_ERROR_ACCESS_DENIED@ 0000000180005fd8     libdatadumpreq001.obj
 0002:00000ff8       ??_C@_0BI@GHECLMNC@JVMTI_ERROR_WRONG_PHASE@ 0000000180005ff8     libdatadumpreq001.obj
 0002:00001010       ??_C@_0BF@OLIHJOII@JVMTI_ERROR_INTERNAL@ 0000000180006010     libdatadumpreq001.obj
 0002:00001028       ??_C@_0BO@EOHGKJHI@JVMTI_ERROR_UNATTACHED_THREAD@ 0000000180006028     libdatadumpreq001.obj
 0002:00001048       ??_C@_0CA@LKHFDACL@JVMTI_ERROR_INVALID_ENVIRONMENT@ 0000000180006048     libdatadumpreq001.obj
 0002:00001068       ??_C@_0BA@MMFHLOKK@?$DMunknown?5error?$DO@ 0000000180006068     libdatadumpreq001.obj
 0002:00001078       ??_C@_0BD@EPBFFECN@JVMTI_PHASE_ONLOAD@ 0000000180006078     libdatadumpreq001.obj
 0002:00001090       ??_C@_0BH@DFOMMNI@JVMTI_PHASE_PRIMORDIAL@ 0000000180006090     libdatadumpreq001.obj
 0002:000010a8       ??_C@_0BC@DEHCLJAD@JVMTI_PHASE_START@ 00000001800060a8     libdatadumpreq001.obj
 0002:000010c0       ??_C@_0BB@CMEPNEPG@JVMTI_PHASE_LIVE@ 00000001800060c0     libdatadumpreq001.obj
 0002:000010d8       ??_C@_0BB@FGJLKEDL@JVMTI_PHASE_DEAD@ 00000001800060d8     libdatadumpreq001.obj
 0002:000010f0       ??_C@_0BA@HPBKJMLO@?$DMunknown?5phase?$DO@ 00000001800060f0     libdatadumpreq001.obj
 0002:00001100       ??_C@_0CF@CBHOKDB@throwable?5?$DN?5jni?9?$DOExceptionOccur@ 0000000180006100     libdatadumpreq001.obj
 0002:00001128       ??_C@_03OFAPEBGM@?$CFs?6@  0000000180006128     libdatadumpreq001.obj
 0002:00001130       ??_C@_0DM@LPIGEGNJ@s?2test?2hotspot?2jtreg?2vmTestbase@ 0000000180006130     libdatadumpreq001.obj
 0002:00001170       ??_C@_0CC@NFCNPEPK@Exception?5in?5JNI?5call?5?$CIcleared?$CJ@ 0000000180006170     libdatadumpreq001.obj
 0002:00001198       ??_C@_0BJ@IBAKFIKF@jni?9?$DOExceptionDescribe?$CI?$CJ@ 0000000180006198     libdatadumpreq001.obj
 0002:000011b8       ??_C@_0BG@GGKALKMH@jni?9?$DOExceptionClear?$CI?$CJ@ 00000001800061b8     libdatadumpreq001.obj
 0002:000011d0       ??_C@_0CF@JMGFGJLJ@?$CD?5?5?5verified?5JNI?5assertion?5is?5F@ 00000001800061d0     libdatadumpreq001.obj
 0002:000011f8       ??_C@_07KBAMPNJK@verbose@  00000001800061f8     libdatadumpreq001.obj
 0002:00001200       ??_C@_0DN@PKJBOLAP@nsk_jvmti_parseOptions?$CI?$CJ?3?5unexp@ 0000000180006200     libdatadumpreq001.obj
 0002:00001240       ??_C@_05IMBNNINJ@trace@    0000000180006240     libdatadumpreq001.obj
 0002:00001248       ??_C@_0DD@BJKGNDMB@nsk_jvmti_parseOptions?$CI?$CJ?3?5no?5va@ 0000000180006248     libdatadumpreq001.obj
 0002:0000127c       ??_C@_04CGFJFPFD@none@     000000018000627c     libdatadumpreq001.obj
 0002:00001284       ??_C@_06BMELKFMA@before@   0000000180006284     libdatadumpreq001.obj
 0002:0000128c       ??_C@_05CMKPCFDK@after@    000000018000628c     libdatadumpreq001.obj
 0002:00001294       ??_C@_03NFKEKGGK@all@      0000000180006294     libdatadumpreq001.obj
 0002:00001298       ??_C@_0DM@NDNJGJKE@nsk_jvmti_parseOptions?$CI?$CJ?3?5uexpe@ 0000000180006298     libdatadumpreq001.obj
 0002:000012d8       ??_C@_08NBBJKJO@waittime@  00000001800062d8     libdatadumpreq001.obj
 0002:000012e8       ??_C@_0DO@CMHGAOHC@nsk_jvmti_parseOptions?$CI?$CJ?3?5not?5i@ 00000001800062e8     libdatadumpreq001.obj
 0002:00001328       ??_C@_0DL@LNMPBDLN@nsk_jvmti_parseOptions?$CI?$CJ?3?5negat@ 0000000180006328     libdatadumpreq001.obj
 0002:00001368       ??_C@_0DA@GMFJNOJH@nsk_jvmti_parseOptions?$CI?$CJ?3?5unkno@ 0000000180006368     libdatadumpreq001.obj
 0002:00001398       ??_C@_0CO@CCIAMEAN@nsk_jvmti_parseOptions?$CI?$CJ?3?5found@ 0000000180006398     libdatadumpreq001.obj
 0002:000013c8       ??_C@_0CJ@OEGPCGDL@nsk_jvmti_parseOptions?$CI?$CJ?3?5out?5o@ 00000001800063c8     libdatadumpreq001.obj
 0002:000013f8       ??_C@_0DI@NMBHPGGF@nsk_jvmti_parseOptions?$CI?$CJ?3?5too?5m@ 00000001800063f8     libdatadumpreq001.obj
 0002:00001430       ??_C@_03POGCGECB@?5?0?$HO@ 0000000180006430     libdatadumpreq001.obj
 0002:00001438       ??_C@_0CB@MLNJNCLJ@?5?5jvmti?5error?3?5code?$DN?$CFd?0?5name?$DN?$CFs@ 0000000180006438     libdatadumpreq001.obj
 0002:00001460       ??_C@_0CD@OHBGDKMK@?$CD?5?5?5jvmti?5error?3?5code?$DN?$CFd?0?5name?$DN@ 0000000180006460     libdatadumpreq001.obj
 0002:00001488       ??_C@_0CG@JNNCGPHB@?$CD?5?5?5error?5expected?3?5code?$DN?$CFd?0?5na@ 0000000180006488     libdatadumpreq001.obj
 0002:000014b0       ??_C@_0EB@IMGKPCGE@?$CIstr_obj?5?$DN?5jni?9?$DONewStringUTF?$CIco@ 00000001800064b0     libdatadumpreq001.obj
 0002:00001500       ??_C@_0EA@HFOGGBCC@s?2test?2hotspot?2jtreg?2vmTestbase@ 0000000180006500     libdatadumpreq001.obj
 0002:00001540       ??_C@_05KKCIMGE@error@     0000000180006540     libdatadumpreq001.obj
 0002:00001548       ??_C@_0BD@HGNAOMCP@agent_data_monitor@ 0000000180006548     libdatadumpreq001.obj
 0002:00001560       ??_C@_0EB@OGCLGKLN@javaVM?9?$DOGetEnv?$CI?$CIvoid?5?$CK?$CK?$CJ?$CGjvmti_@ 0000000180006560     libdatadumpreq001.obj
 0002:000015b0       ??_C@_0EA@PNBCDMOA@s?2test?2hotspot?2jtreg?2vmTestbase@ 00000001800065b0     libdatadumpreq001.obj
 0002:000015f0       ??_C@_0CI@DDPIFBGM@init_agent_data?$CIjvmti_env?0?5?$CGage@ 00000001800065f0     libdatadumpreq001.obj
 0002:00001618       ??_C@_0DI@ILAHDLMP@?$CI?$CKagentThreadProc?$CJ?$CIjvmti_env?0?5a@ 0000000180006618     libdatadumpreq001.obj
 0002:00001650       ??_C@_0BD@KDBALNLB@JVMTI?5agent?5thread@ 0000000180006650     libdatadumpreq001.obj
 0002:00001668       ??_C@_0BB@NOKBFPFO@java?1lang?1Thread@ 0000000180006668     libdatadumpreq001.obj
 0002:0000167c       ??_C@_06FALKBLGB@?$DMinit?$DO@ 000000018000667c     libdatadumpreq001.obj
 0002:00001688       ??_C@_0BG@IKDDPPGD@?$CILjava?1lang?1String?$DL?$CJV@ 0000000180006688     libdatadumpreq001.obj
 0002:000016a0       ??_C@_0EB@IFJBFEKC@?$CIthreadClass?5?$DN?5jni_env?9?$DOFindCla@ 00000001800066a0     libdatadumpreq001.obj
 0002:000016f0       ??_C@_0GF@FGFIBKKL@?$CIthreadCtor?5?$DN?5jni_env?9?$DOGetMetho@ 00000001800066f0     libdatadumpreq001.obj
 0002:00001758       ??_C@_0DN@NCPDJLOG@?$CIthreadName?5?$DN?5jni_env?9?$DONewStrin@ 0000000180006758     libdatadumpreq001.obj
 0002:000017a0       ??_C@_0FE@PFKODBGC@?$CIthreadObject?5?$DN?5jni_env?9?$DONewObj@ 00000001800067a0     libdatadumpreq001.obj
 0002:00001800       ??_C@_0ED@HOBAHHJI@?$CIthreadGlobalRef?5?$DN?5jni_env?9?$DONew@ 0000000180006800     libdatadumpreq001.obj
 0002:00001850       ??_C@_0FN@HNJJAHFC@jvmti_env?9?$DORunAgentThread?$CIagent@ 0000000180006850     libdatadumpreq001.obj
 0002:000018b0       ??_C@_0EA@MOJDNKDF@Debuggee?5status?5sync?5aborted?5be@ 00000001800068b0     libdatadumpreq001.obj
 0002:000018f0       ??_C@_0EA@EEOEJAEN@status?5?$DN?5syncDebuggeeStatus?$CIjni@ 00000001800068f0     libdatadumpreq001.obj
 0002:00001930       ??_C@_0BL@JBCFNBMB@nsk_jvmti_resetAgentData?$CI?$CJ@ 0000000180006930     libdatadumpreq001.obj
 0002:00001950       ??_C@_0EL@LPBEELIP@s?2test?2hotspot?2jtreg?2vmTestbase@ 0000000180006950     libdatadumpreq001.obj
 0002:000019a0       ??_C@_0CK@JDAMFDMJ@jvmti?9?$DOSetTag?$CIo?0?5tag?$CJ?5?$DN?$DN?5JVMTI_@ 00000001800069a0     libdatadumpreq001.obj
 0002:000019d0       ??_C@_0CC@DAMNHKNI@Can?8t?5set?5tag?5?$CFli?5for?5object?5?$CFl@ 00000001800069d0     libdatadumpreq001.obj
 0002:000019f8       ??_C@_0DL@HAJPNKEF@jvmti?9?$DOGetObjectHashCode?$CIo?0?5?$CGha@ 00000001800069f8     libdatadumpreq001.obj
 0002:00001a38       ??_C@_0BL@JFPIEOBF@Can?8t?5get?5hash?5object?5?$CFlx?6@ 0000000180006a38     libdatadumpreq001.obj
 0002:00001a58       ??_C@_0BG@DICPHBKN@setTag?3?5?$CF08x?5?$DM?9?5?$CF?53li@ 0000000180006a58     libdatadumpreq001.obj
 0002:00001a70       ??_C@_0DH@FCEEBDMJ@?$CIs?5?$DN?5jni?9?$DOGetStringUTFChars?$CIsIn@ 0000000180006a70     libdatadumpreq001.obj
 0002:00001aa8       ??_C@_0BJ@OKKGHDCN@Can?8t?5get?5string?5at?5?$CF?$CDp?6@ 0000000180006aa8     libdatadumpreq001.obj
 0002:00001ac8       ??_C@_0BP@EKFLGGFJ@Can?8t?5get?5string?5at?5?$CF?$CDp?3?5null?6@ 0000000180006ac8     libdatadumpreq001.obj
 0002:00001ae8       ??_C@_06ICODBHCL@?5?1?1?5?$CFs@ 0000000180006ae8     libdatadumpreq001.obj
 0002:00001af0       ??_C@_0DB@KGFPLEGO@?$CIr?5?$DN?5jvmti?9?$DOGetTag?$CIo?0?5?$CGtag?$CJ?$CJ?5?$DN?$DN@ 0000000180006af0     libdatadumpreq001.obj
 0002:00001b28       ??_C@_0CO@PDAGBCGJ@Can?8t?5GetTag?5for?5object?5?$CFlx?4?5Re@ 0000000180006b28     libdatadumpreq001.obj
 0002:00001b58       ??_C@_0CH@HPEODOHC@TEST_BUG?3?5Max?4?5number?5of?5refs?5r@ 0000000180006b58     libdatadumpreq001.obj
 0002:00001b80       ??_C@_0DI@PHFCABIM@?$CIr?5?$DN?5jvmti?9?$DOGetTag?$CIfrom?0?5?$CGtagFr@ 0000000180006b80     libdatadumpreq001.obj
 0002:00001bb8       ??_C@_0DI@MDEGFNKD@TEST_BUG?3?5Can?8t?5GetTag?5for?5obje@ 0000000180006bb8     libdatadumpreq001.obj
 0002:00001bf0       ??_C@_0DE@MLELJAHM@?$CIr?5?$DN?5jvmti?9?$DOGetTag?$CIto?0?5?$CGtagTo?$CJ?$CJ@ 0000000180006bf0     libdatadumpreq001.obj
 0002:00001c28       ??_C@_0CF@HCFBMNJF@?$DO?$DO?$DO?$DO?5DataDumpRequest?5event?5rece@ 0000000180006c28     libdatadumpreq001.obj
 0002:00001c50       ??_C@_0FM@KAJPEGCE@s?2test?2hotspot?2jtreg?2vmTestbase@ 0000000180006c50     libdatadumpreq001.obj
 0002:00001cb0       ??_C@_0EG@DDHFKJLI@TEST?5FAILED?3?5DataDumpRequest?5ev@ 0000000180006cb0     libdatadumpreq001.obj
 0002:00001d00       ??_C@_0FA@GMHBBHJF@CHECK?5PASSED?3?5DataDumpRequest?5e@ 0000000180006d00     libdatadumpreq001.obj
 0002:00001d50       ??_C@_06FHLMFHLD@?$DM?$DM?$DM?$DM?6?6@ 0000000180006d50     libdatadumpreq001.obj
 0002:00001d58       ??_C@_0CG@OAEACOCP@waiting?5for?5DataDumpRequest?5eve@ 0000000180006d58     libdatadumpreq001.obj
 0002:00001d80       ??_C@_0CA@MNKGCBCG@nsk_jvmti_parseOptions?$CIoptions?$CJ@ 0000000180006d80     libdatadumpreq001.obj
 0002:00001da0       ??_C@_0BB@CGPOECH@jvmti?5?$CB?$DN?5nullptr@ 0000000180006da0     libdatadumpreq001.obj
 0002:00001db8       ??_C@_0BK@BCOFKMHD@data?5dump?5request?5monitor@ 0000000180006db8     libdatadumpreq001.obj
 0002:00001dd8       ??_C@_0BN@HGIKGGD@setting?5event?5callbacks?5?4?4?4?6@ 0000000180006dd8     libdatadumpreq001.obj
 0002:00001df8       ??_C@_0DI@NJCFGEGC@jvmti?9?$DOSetEventCallbacks?$CI?$CGcallb@ 0000000180006df8     libdatadumpreq001.obj
 0002:00001e30       ??_C@_0DI@LEFDPPF@setting?5event?5callbacks?5done?6en@ 0000000180006e30     libdatadumpreq001.obj
 0002:00001e70       ??_C@_0FG@KGGAGOKN@jvmti?9?$DOSetEventNotificationMode@ 0000000180006e70     libdatadumpreq001.obj
 0002:00001ec8       ??_C@_0BL@GBOGNFCP@enabling?5the?5events?5done?6?6@ 0000000180006ec8     libdatadumpreq001.obj
 0002:00001f00       ??_C@_1EC@JIJBPKFM@?$AAa?$AAp?$AAi?$AA?9?$AAm?$AAs?$AA?9?$AAw?$AAi?$AAn?$AA?9?$AAc?$AAo?$AAr?$AAe@ 0000000180006f00     MSVCRT:thread_safe_statics.obj
 0002:00001f48       ??_C@_1BK@MGMFAEKH@?$AAk?$AAe?$AAr?$AAn?$AAe?$AAl?$AA3?$AA2?$AA?4?$AAd?$AAl?$AAl@ 0000000180006f48     MSVCRT:thread_safe_statics.obj
 0002:00001f68       ??_C@_0BJ@JEBJOJFJ@SleepConditionVariableCS@ 0000000180006f68     MSVCRT:thread_safe_statics.obj
 0002:00001f88       ??_C@_0BJ@PGPPEPCC@WakeAllConditionVariable@ 0000000180006f88     MSVCRT:thread_safe_statics.obj
 0002:00001fa8       _pDefaultRawDllMain        0000000180006fa8     MSVCRT:dll_dllmain.obj
 0002:00001fa8       _pRawDllMain               0000000180006fa8     MSVCRT:dll_dllmain.obj
 0002:00001fb0       __xmm@ffffffffffffffffffffffffffffffff 0000000180006fb0     MSVCRT:utility.obj
 0002:00001fc0       _load_config_used          0000000180006fc0     MSVCRT:loadcfg.obj
 0002:00002180       _tls_used                  0000000180007180     MSVCRT:tlssup.obj
 0002:000021a8       __volatile_metadata        00000001800071a8     <linker-defined>
 0002:00002580       __rtc_iaa                  0000000180007580     MSVCRT:initsect.obj
 0002:00002588       __rtc_izz                  0000000180007588     MSVCRT:initsect.obj
 0002:00002590       __rtc_taa                  0000000180007590     MSVCRT:initsect.obj
 0002:00002598       __rtc_tzz                  0000000180007598     MSVCRT:initsect.obj
 0002:000025a0       _tls_start                 00000001800075a0     MSVCRT:tlssup.obj
 0002:000025a4       _Init_thread_epoch         00000001800075a4     MSVCRT:thread_safe_statics.obj
 0002:000025a8       _tls_end                   00000001800075a8     MSVCRT:tlssup.obj
 0002:00002c8c       __IMPORT_DESCRIPTOR_KERNEL32 0000000180007c8c     kernel32:KERNEL32.dll
 0002:00002ca0       __IMPORT_DESCRIPTOR_VCRUNTIME140 0000000180007ca0     vcruntime:VCRUNTIME140.dll
 0002:00002cb4       __IMPORT_DESCRIPTOR_api-ms-win-crt-heap-l1-1-0 0000000180007cb4     ucrt:api-ms-win-crt-heap-l1-1-0.dll
 0002:00002cc8       __IMPORT_DESCRIPTOR_api-ms-win-crt-runtime-l1-1-0 0000000180007cc8     ucrt:api-ms-win-crt-runtime-l1-1-0.dll
 0002:00002cdc       __IMPORT_DESCRIPTOR_api-ms-win-crt-convert-l1-1-0 0000000180007cdc     ucrt:api-ms-win-crt-convert-l1-1-0.dll
 0002:00002cf0       __IMPORT_DESCRIPTOR_api-ms-win-crt-stdio-l1-1-0 0000000180007cf0     ucrt:api-ms-win-crt-stdio-l1-1-0.dll
 0002:00002d04       __IMPORT_DESCRIPTOR_api-ms-win-crt-string-l1-1-0 0000000180007d04     ucrt:api-ms-win-crt-string-l1-1-0.dll
 0002:00002d18       __NULL_IMPORT_DESCRIPTOR   0000000180007d18     kernel32:KERNEL32.dll
 0003:00000034       _Init_global_epoch         0000000180009034     MSVCRT:thread_safe_statics.obj
 0003:00000040       __security_cookie          0000000180009040     MSVCRT:gs_cookie.obj
 0003:00000048       __security_cookie_complement 0000000180009048     MSVCRT:gs_cookie.obj
 0003:00000050       __scrt_native_dllmain_reason 0000000180009050     MSVCRT:utility.obj
 0003:00000058       __isa_available            0000000180009058     MSVCRT:cpu_disp.obj
 0003:0000005c       __isa_enabled              000000018000905c     MSVCRT:cpu_disp.obj
 0003:00000060       __memset_fast_string_threshold 0000000180009060     MSVCRT:cpu_disp.obj
 0003:00000068       __memset_nt_threshold      0000000180009068     MSVCRT:cpu_disp.obj
 0003:00000070       __scrt_ucrt_dll_is_in_use  0000000180009070     MSVCRT:ucrt_stubs.obj
 0003:00000080       g_wrongHeapCallbacks       0000000180009080     libdatadumpreq001.obj
 0003:00000100       g_szTagInfo                0000000180009100     libdatadumpreq001.obj
 0003:00002040       g_tagFlags                 000000018000b040     libdatadumpreq001.obj
 0003:00002428       g_refsToVerifyCnt          000000018000b428     libdatadumpreq001.obj
 0003:0000242c       g_fakeUserData             000000018000b42c     libdatadumpreq001.obj
 0003:00002430       g_tagVisitCount            000000018000b430     libdatadumpreq001.obj
 0003:000033d0       g_refsToVerify             000000018000c3d0     libdatadumpreq001.obj
 0003:0001aad0       g_userDataError            0000000180023ad0     libdatadumpreq001.obj
 0003:0001adb0       ?_OptionsStorage@?1??__local_stdio_printf_options@@9@4_KA 0000000180023db0     libdatadumpreq001.obj
 0003:0001b378       _tls_index                 0000000180024378     MSVCRT:tlssup.obj
 0003:0001b380       __scrt_current_native_startup_state 0000000180024380     MSVCRT:utility.obj
 0003:0001b388       __scrt_native_startup_lock 0000000180024388     MSVCRT:utility.obj
 0003:0001b3c8       __scrt_debugger_hook_flag  00000001800243c8     MSVCRT:utility_desktop.obj
 0003:0001b3d0       ?__type_info_root_node@@3U__type_info_node@@A 00000001800243d0     MSVCRT:tncleanup.obj
 0003:0001b3e0       ?_OptionsStorage@?1??__local_stdio_scanf_options@@9@4_KA 00000001800243e0     MSVCRT:default_local_stdio_options.obj
 0003:0001b3e8       __favor                    00000001800243e8     MSVCRT:cpu_disp.obj
 0003:0001b3f0       __dyn_tls_init_callback    00000001800243f0     <common>

 entry point at        0001:000029b0

 Static symbols

 0000:fffd9000       .debug$S                   0000000180000000     datadumpreq001.exp
 0000:fffd9000       .debug$S                   0000000180000000     vcruntime:VCRUNTIME140.dll
 0000:fffd9000       .debug$S                   0000000180000000     vcruntime:VCRUNTIME140.dll
 0000:fffd9000       .debug$S                   0000000180000000     vcruntime:VCRUNTIME140.dll
 0000:fffd9000       .debug$S                   0000000180000000     vcruntime:VCRUNTIME140.dll
 0000:fffd9000       .debug$S                   0000000180000000     vcruntime:VCRUNTIME140.dll
 0000:fffd9000       .debug$S                   0000000180000000     vcruntime:VCRUNTIME140.dll
 0000:fffd9000       .debug$S                   0000000180000000     vcruntime:VCRUNTIME140.dll
 0000:fffd9000       .debug$S                   0000000180000000     ucrt:api-ms-win-crt-convert-l1-1-0.dll
 0000:fffd9000       .debug$S                   0000000180000000     ucrt:api-ms-win-crt-heap-l1-1-0.dll
 0000:fffd9000       .debug$S                   0000000180000000     ucrt:api-ms-win-crt-heap-l1-1-0.dll
 0000:fffd9000       .debug$S                   0000000180000000     ucrt:api-ms-win-crt-heap-l1-1-0.dll
 0000:fffd9000       .debug$S                   0000000180000000     ucrt:api-ms-win-crt-heap-l1-1-0.dll
 0000:fffd9000       .debug$S                   0000000180000000     ucrt:api-ms-win-crt-runtime-l1-1-0.dll
 0000:fffd9000       .debug$S                   0000000180000000     ucrt:api-ms-win-crt-runtime-l1-1-0.dll
 0000:fffd9000       .debug$S                   0000000180000000     ucrt:api-ms-win-crt-runtime-l1-1-0.dll
 0000:fffd9000       .debug$S                   0000000180000000     ucrt:api-ms-win-crt-runtime-l1-1-0.dll
 0000:fffd9000       .debug$S                   0000000180000000     ucrt:api-ms-win-crt-runtime-l1-1-0.dll
 0000:fffd9000       .debug$S                   0000000180000000     ucrt:api-ms-win-crt-runtime-l1-1-0.dll
 0000:fffd9000       .debug$S                   0000000180000000     ucrt:api-ms-win-crt-runtime-l1-1-0.dll
 0000:fffd9000       .debug$S                   0000000180000000     ucrt:api-ms-win-crt-runtime-l1-1-0.dll
 0000:fffd9000       .debug$S                   0000000180000000     ucrt:api-ms-win-crt-runtime-l1-1-0.dll
 0000:fffd9000       .debug$S                   0000000180000000     ucrt:api-ms-win-crt-runtime-l1-1-0.dll
 0000:fffd9000       .debug$S                   0000000180000000     ucrt:api-ms-win-crt-runtime-l1-1-0.dll
 0000:fffd9000       .debug$S                   0000000180000000     ucrt:api-ms-win-crt-runtime-l1-1-0.dll
 0000:fffd9000       .debug$S                   0000000180000000     ucrt:api-ms-win-crt-runtime-l1-1-0.dll
 0000:fffd9000       .debug$S                   0000000180000000     ucrt:api-ms-win-crt-runtime-l1-1-0.dll
 0000:fffd9000       .debug$S                   0000000180000000     ucrt:api-ms-win-crt-runtime-l1-1-0.dll
 0000:fffd9000       .debug$S                   0000000180000000     ucrt:api-ms-win-crt-runtime-l1-1-0.dll
 0000:fffd9000       .debug$S                   0000000180000000     ucrt:api-ms-win-crt-stdio-l1-1-0.dll
 0000:fffd9000       .debug$S                   0000000180000000     ucrt:api-ms-win-crt-stdio-l1-1-0.dll
 0000:fffd9000       .debug$S                   0000000180000000     ucrt:api-ms-win-crt-stdio-l1-1-0.dll
 0000:fffd9000       .debug$S                   0000000180000000     ucrt:api-ms-win-crt-stdio-l1-1-0.dll
 0000:fffd9000       .debug$S                   0000000180000000     ucrt:api-ms-win-crt-stdio-l1-1-0.dll
 0000:fffd9000       .debug$S                   0000000180000000     ucrt:api-ms-win-crt-stdio-l1-1-0.dll
 0000:fffd9000       .debug$S                   0000000180000000     ucrt:api-ms-win-crt-stdio-l1-1-0.dll
 0000:fffd9000       .debug$S                   0000000180000000     ucrt:api-ms-win-crt-stdio-l1-1-0.dll
 0000:fffd9000       .debug$S                   0000000180000000     ucrt:api-ms-win-crt-stdio-l1-1-0.dll
 0000:fffd9000       .debug$S                   0000000180000000     ucrt:api-ms-win-crt-stdio-l1-1-0.dll
 0000:fffd9000       .debug$S                   0000000180000000     ucrt:api-ms-win-crt-string-l1-1-0.dll
 0000:fffd9000       .debug$S                   0000000180000000     ucrt:api-ms-win-crt-string-l1-1-0.dll
 0000:fffd9000       .debug$S                   0000000180000000     ucrt:api-ms-win-crt-string-l1-1-0.dll
 0000:fffd9000       .debug$S                   0000000180000000     ucrt:api-ms-win-crt-string-l1-1-0.dll
 0000:fffd9000       .debug$S                   0000000180000000     ucrt:api-ms-win-crt-string-l1-1-0.dll
 0000:fffd9000       .debug$S                   0000000180000000     ucrt:api-ms-win-crt-string-l1-1-0.dll
 0000:fffd9000       .debug$S                   0000000180000000     ucrt:api-ms-win-crt-string-l1-1-0.dll
 0000:fffd9000       .debug$S                   0000000180000000     ucrt:api-ms-win-crt-string-l1-1-0.dll
 0000:fffd9000       .debug$S                   0000000180000000     kernel32:KERNEL32.dll
 0000:fffd9000       .debug$S                   0000000180000000     kernel32:KERNEL32.dll
 0000:fffd9000       .debug$S                   0000000180000000     kernel32:KERNEL32.dll
 0000:fffd9000       .debug$S                   0000000180000000     kernel32:KERNEL32.dll
 0000:fffd9000       .debug$S                   0000000180000000     kernel32:KERNEL32.dll
 0000:fffd9000       .debug$S                   0000000180000000     kernel32:KERNEL32.dll
 0000:fffd9000       .debug$S                   0000000180000000     kernel32:KERNEL32.dll
 0000:fffd9000       .debug$S                   0000000180000000     kernel32:KERNEL32.dll
 0000:fffd9000       .debug$S                   0000000180000000     kernel32:KERNEL32.dll
 0000:fffd9000       .debug$S                   0000000180000000     kernel32:KERNEL32.dll
 0000:fffd9000       .debug$S                   0000000180000000     kernel32:KERNEL32.dll
 0000:fffd9000       .debug$S                   0000000180000000     kernel32:KERNEL32.dll
 0000:fffd9000       .debug$S                   0000000180000000     kernel32:KERNEL32.dll
 0000:fffd9000       .debug$S                   0000000180000000     kernel32:KERNEL32.dll
 0000:fffd9000       .debug$S                   0000000180000000     kernel32:KERNEL32.dll
 0000:fffd9000       .debug$S                   0000000180000000     kernel32:KERNEL32.dll
 0000:fffd9000       .debug$S                   0000000180000000     kernel32:KERNEL32.dll
 0000:fffd9000       .debug$S                   0000000180000000     kernel32:KERNEL32.dll
 0000:fffd9000       .debug$S                   0000000180000000     kernel32:KERNEL32.dll
 0000:fffd9000       .debug$S                   0000000180000000     kernel32:KERNEL32.dll
 0000:fffd9000       .debug$S                   0000000180000000     kernel32:KERNEL32.dll
 0000:fffd9000       .debug$S                   0000000180000000     kernel32:KERNEL32.dll
 0000:fffd9000       .debug$S                   0000000180000000     kernel32:KERNEL32.dll
 0000:fffd9000       .debug$S                   0000000180000000     kernel32:KERNEL32.dll
 0000:fffd9000       .debug$S                   0000000180000000     kernel32:KERNEL32.dll
 0000:fffd9000       .debug$S                   0000000180000000     kernel32:KERNEL32.dll
 0000:fffd9000       .debug$S                   0000000180000000     kernel32:KERNEL32.dll
 0000:fffd9000       .debug$S                   0000000180000000     kernel32:KERNEL32.dll
 0001:00000754       DataDumpRequest            0000000180001754 f   libdatadumpreq001.obj
 0001:00001054       addRefToVerify             0000000180002054 f   libdatadumpreq001.obj
 0001:000010c8       agentThreadWrapper         00000001800020c8 f   libdatadumpreq001.obj
 0001:0000121c       check_option               000000018000221c f   libdatadumpreq001.obj
 0001:000014ec       file_basename              00000001800024ec f   libdatadumpreq001.obj
 0001:00001ec0       startAgentThreadWrapper    0000000180002ec0 f   libdatadumpreq001.obj
 0001:000021ec       syncDebuggeeStatus         00000001800031ec f   libdatadumpreq001.obj
 0001:00002474       capture_previous_context   0000000180003474 f   MSVCRT:gs_report.obj
 0001:000024e8       ?__scrt_initialize_thread_safe_statics@@YAHXZ 00000001800034e8 f   MSVCRT:thread_safe_statics.obj
 0001:000025b8       ?__scrt_uninitialize_thread_safe_statics@@YAXXZ 00000001800035b8 f   MSVCRT:thread_safe_statics.obj
 0001:00002660       $$000000                   0000000180003660     MSVCRT:amdsecgs.obj
 0001:00002690       ?dllmain_crt_dispatch@@YAHQEAUHINSTANCE__@@KQEAX@Z 0000000180003690 f   MSVCRT:dll_dllmain.obj
 0001:000026e0       ?dllmain_crt_process_attach@@YAHQEAUHINSTANCE__@@QEAX@Z 00000001800036e0 f   MSVCRT:dll_dllmain.obj
 0001:000027f8       ?dllmain_crt_process_detach@@YAH_N@Z 00000001800037f8 f   MSVCRT:dll_dllmain.obj
 0001:0000287c       ?dllmain_dispatch@@YAHQEAUHINSTANCE__@@KQEAX@Z 000000018000387c f   MSVCRT:dll_dllmain.obj
 0001:00003290       $$000000                   0000000180004290     MSVCRT:guard_dispatch.obj
 0001:000032b0       $$000000                   00000001800042b0     MSVCRT:guard_xfg_dispatch.obj
 0001:000032c6       ?fin$0@?0??dllmain_crt_process_attach@@YAHQEAUHINSTANCE__@@QEAX@Z@4HA 00000001800042c6 f   MSVCRT:dll_dllmain.obj
 0001:000032dd       ?fin$0@?0??dllmain_crt_process_detach@@YAH_N@Z@4HA 00000001800042dd f   MSVCRT:dll_dllmain.obj
 0001:000032f6       ?fin$1@?0??dllmain_crt_process_detach@@YAH_N@Z@4HA 00000001800042f6 f   MSVCRT:dll_dllmain.obj
 0001:0000330a       ?filt$0@?0??dllmain_dispatch@@YAHQEAUHINSTANCE__@@KQEAX@Z@4HA 000000018000430a f   MSVCRT:dll_dllmain.obj
 0001:00003340       __scrt_is_nonwritable_in_current_image$filt$0 0000000180004340 f   MSVCRT:utility.obj
 0002:00000218       ?__scrt_initialize_tss_var@@3P6AHXZEA 0000000180005218     MSVCRT:thread_safe_statics.obj
 0002:00000340       ?opcLengths@@3QBEB         0000000180005340     libdatadumpreq001.obj
 0002:00001ee8       GS_ExceptionPointers       0000000180006ee8     MSVCRT:gs_report.obj
 0002:000025b0       $unwind$fprintf            00000001800075b0     libdatadumpreq001.obj
 0002:000025bc       $unwind$printf             00000001800075bc     libdatadumpreq001.obj
 0002:000025c8       $unwind$?NewObject@JNIEnv_@@QEAAPEAV_jobject@@PEAV_jclass@@PEAU_jmethodID@@ZZ 00000001800075c8     libdatadumpreq001.obj
 0002:000025c8       $unwind$nsk_lcomplain      00000001800075c8     libdatadumpreq001.obj
 0002:000025c8       $unwind$nsk_ldisplay       00000001800075c8     libdatadumpreq001.obj
 0002:000025d0       $unwind$nsk_lvdisplay      00000001800075d0     libdatadumpreq001.obj
 0002:000025d0       $unwind$_RTC_Initialize    00000001800075d0     MSVCRT:initsect.obj
 0002:000025d0       $unwind$_RTC_Terminate     00000001800075d0     MSVCRT:initsect.obj
 0002:000025d0       $unwind$?__scrt_initialize_thread_safe_statics@@YAHXZ 00000001800075d0     MSVCRT:thread_safe_statics.obj
 0002:000025dc       $unwind$nsk_complain       00000001800075dc     libdatadumpreq001.obj
 0002:000025dc       $unwind$nsk_printf         00000001800075dc     libdatadumpreq001.obj
 0002:000025e4       $unwind$nsk_lvcomplain     00000001800075e4     libdatadumpreq001.obj
 0002:000025fc       $unwind$nsk_ltrace         00000001800075fc     libdatadumpreq001.obj
 0002:000025fc       $unwind$__report_gsfailure 00000001800075fc     MSVCRT:gs_report.obj
 0002:00002604       $unwind$DataDumpRequest    0000000180007604     libdatadumpreq001.obj
 0002:00002604       $unwind$Java_nsk_jvmti_DataDumpRequest_datadumpreq001_waitForResult 0000000180007604     libdatadumpreq001.obj
 0002:00002604       $unwind$nsk_lvtrace        0000000180007604     libdatadumpreq001.obj
 0002:00002604       $unwind$__raise_securityfailure 0000000180007604     MSVCRT:gs_report.obj
 0002:00002604       $unwind$__scrt_initialize_crt 0000000180007604     MSVCRT:utility.obj
 0002:00002604       $unwind$__scrt_initialize_onexit_tables 0000000180007604     MSVCRT:utility.obj
 0002:00002604       $unwind$__scrt_release_startup_lock 0000000180007604     MSVCRT:utility.obj
 0002:00002604       $unwind$__scrt_uninitialize_crt 0000000180007604     MSVCRT:utility.obj
 0002:00002604       $unwind$_onexit            0000000180007604     MSVCRT:utility.obj
 0002:0000260c       $unwind$nsk_lverify        000000018000760c     libdatadumpreq001.obj
 0002:0000261c       $unwind$nsk_vprintf        000000018000761c     libdatadumpreq001.obj
 0002:0000262c       $unwind$?nsk_jni_lverify@@YAHHPEAUJNIEnv_@@HQEBDH1ZZ 000000018000762c     libdatadumpreq001.obj
 0002:00002640       $unwind$?nsk_jni_check_exception@@YAHPEAUJNIEnv_@@QEBDH@Z 0000000180007640     libdatadumpreq001.obj
 0002:0000265c       $unwind$nsk_jvmti_parseOptions 000000018000765c     libdatadumpreq001.obj
 0002:00002678       $unwind$nsk_jvmti_createJVMTIEnv 0000000180007678     libdatadumpreq001.obj
 0002:0000268c       $unwind$Java_nsk_jvmti_unit_FollowReferences_FollowRefObjects_resetTags 000000018000768c     libdatadumpreq001.obj
 0002:0000268c       $unwind$addRefToVerify     000000018000768c     libdatadumpreq001.obj
 0002:0000268c       $unwind$nsk_jvmti_resetAgentData 000000018000768c     libdatadumpreq001.obj
 0002:0000268c       $unwind$__scrt_initialize_default_local_stdio_options 000000018000768c     MSVCRT:default_local_stdio_options.obj
 0002:0000268c       $unwind$?dllmain_crt_dispatch@@YAHQEAUHINSTANCE__@@KQEAX@Z 000000018000768c     MSVCRT:dll_dllmain.obj
 0002:0000268c       $unwind$DllMain            000000018000768c     MSVCRT:dll_dllmain_stub.obj
 0002:0000268c       $unwind$__GSHandlerCheck   000000018000768c     MSVCRT:gshandler.obj
 0002:0000268c       $unwind$?__scrt_uninitialize_thread_safe_statics@@YAXXZ 000000018000768c     MSVCRT:thread_safe_statics.obj
 0002:0000268c       $unwind$__scrt_acquire_startup_lock 000000018000768c     MSVCRT:utility.obj
 0002:0000268c       $unwind$__scrt_dllmain_after_initialize_c 000000018000768c     MSVCRT:utility.obj
 0002:0000268c       $unwind$__scrt_dllmain_before_initialize_c 000000018000768c     MSVCRT:utility.obj
 0002:0000268c       $unwind$__scrt_dllmain_crt_thread_attach 000000018000768c     MSVCRT:utility.obj
 0002:0000268c       $unwind$__scrt_dllmain_crt_thread_detach 000000018000768c     MSVCRT:utility.obj
 0002:0000268c       $unwind$__scrt_dllmain_uninitialize_c 000000018000768c     MSVCRT:utility.obj
 0002:0000268c       $unwind$__scrt_dllmain_uninitialize_critical 000000018000768c     MSVCRT:utility.obj
 0002:0000268c       $unwind$atexit             000000018000768c     MSVCRT:utility.obj
 0002:00002694       $unwind$nsk_jvmti_lverify  0000000180007694     libdatadumpreq001.obj
 0002:000026a8       $unwind$createRawMonitor   00000001800076a8     libdatadumpreq001.obj
 0002:000026b8       $unwind$exitOnError        00000001800076b8     libdatadumpreq001.obj
 0002:000026c8       $unwind$check_option       00000001800076c8     libdatadumpreq001.obj
 0002:000026c8       $unwind$_DllMainCRTStartup 00000001800076c8     MSVCRT:dll_dllmain.obj
 0002:000026d8       $unwind$Java_nsk_share_jvmti_ArgumentHandler_getAgentOptionsString 00000001800076d8     libdatadumpreq001.obj
 0002:000026ec       $unwind$Java_nsk_jvmti_unit_FollowReferences_FollowRefObjects_getTag 00000001800076ec     libdatadumpreq001.obj
 0002:000026ec       $unwind$Java_nsk_share_jvmti_DebugeeClass_checkStatus 00000001800076ec     libdatadumpreq001.obj
 0002:000026ec       $unwind$agentThreadWrapper 00000001800076ec     libdatadumpreq001.obj
 0002:000026fc       $unwind$startAgentThreadWrapper 00000001800076fc     libdatadumpreq001.obj
 0002:00002718       $unwind$syncDebuggeeStatus 0000000180007718     libdatadumpreq001.obj
 0002:00002718       $unwind$__scrt_dllmain_exception_filter 0000000180007718     MSVCRT:utility.obj
 0002:0000272c       $unwind$Java_nsk_share_jvmti_DebugeeClass_resetAgentData 000000018000772c     libdatadumpreq001.obj
 0002:00002734       $unwind$MA_checkStatus     0000000180007734     libdatadumpreq001.obj
 0002:00002748       $unwind$Java_nsk_jvmti_unit_FollowReferences_FollowRefObjects_setTag 0000000180007748     libdatadumpreq001.obj
 0002:00002760       $unwind$Java_nsk_jvmti_unit_FollowReferences_FollowRefObjects_addRefToVerify 0000000180007760     libdatadumpreq001.obj
 0002:0000277c       $unwind$Agent_Initialize   000000018000777c     libdatadumpreq001.obj
 0002:00002798       $unwind$capture_previous_context 0000000180007798     MSVCRT:gs_report.obj
 0002:000027a4       $unwind$__GSHandlerCheckCommon 00000001800077a4     MSVCRT:gshandler.obj
 0002:000027b0       $xdatasym                  00000001800077b0     MSVCRT:amdsecgs.obj
 0002:000027b4       $unwind$?dllmain_crt_process_attach@@YAHQEAUHINSTANCE__@@QEAX@Z 00000001800077b4     MSVCRT:dll_dllmain.obj
 0002:000027f0       $unwind$?fin$0@?0??dllmain_crt_process_attach@@YAHQEAUHINSTANCE__@@QEAX@Z@4HA 00000001800077f0     MSVCRT:dll_dllmain.obj
 0002:000027f0       $unwind$?fin$0@?0??dllmain_crt_process_detach@@YAH_N@Z@4HA 00000001800077f0     MSVCRT:dll_dllmain.obj
 0002:000027f0       $unwind$?fin$1@?0??dllmain_crt_process_detach@@YAH_N@Z@4HA 00000001800077f0     MSVCRT:dll_dllmain.obj
 0002:000027f8       $unwind$?dllmain_crt_process_detach@@YAH_N@Z 00000001800077f8     MSVCRT:dll_dllmain.obj
 0002:0000284c       $unwind$?dllmain_dispatch@@YAHQEAUHINSTANCE__@@KQEAX@Z 000000018000784c     MSVCRT:dll_dllmain.obj
 0002:00002874       $unwind$?filt$0@?0??dllmain_dispatch@@YAHQEAUHINSTANCE__@@KQEAX@Z@4HA 0000000180007874     MSVCRT:dll_dllmain.obj
 0002:0000287c       $unwind$__scrt_is_nonwritable_in_current_image 000000018000787c     MSVCRT:utility.obj
 0002:0000289c       $unwind$__scrt_is_nonwritable_in_current_image$filt$0 000000018000789c     MSVCRT:utility.obj
 0002:000028a4       $unwind$__scrt_fastfail    00000001800078a4     MSVCRT:utility_desktop.obj
 0002:000028b4       $unwind$__security_init_cookie 00000001800078b4     MSVCRT:gs_support.obj
 0002:000028c0       $unwind$__isa_available_init 00000001800078c0     MSVCRT:cpu_disp.obj
 0002:000028d0       $xdatasym                  00000001800078d0     MSVCRT:guard_dispatch.obj
 0002:000028d8       $xdatasym                  00000001800078d8     MSVCRT:guard_xfg_dispatch.obj
 0002:000028e0       .edata                     00000001800078e0     datadumpreq001.exp
 0002:00002908       rgpv                       0000000180007908     datadumpreq001.exp
 0002:00002944       rgszName                   0000000180007944     datadumpreq001.exp
 0002:00002980       rgwOrd                     0000000180007980     datadumpreq001.exp
 0002:0000299e       szName                     000000018000799e     datadumpreq001.exp
 0002:000029b1       $N00001                    00000001800079b1     datadumpreq001.exp
 0002:000029c0       $N00002                    00000001800079c0     datadumpreq001.exp
 0002:000029cd       $N00003                    00000001800079cd     datadumpreq001.exp
 0002:00002a09       $N00004                    0000000180007a09     datadumpreq001.exp
 0002:00002a4e       $N00005                    0000000180007a4e     datadumpreq001.exp
 0002:00002a8b       $N00006                    0000000180007a8b     datadumpreq001.exp
 0002:00002ad3       $N00007                    0000000180007ad3     datadumpreq001.exp
 0002:00002b13       $N00008                    0000000180007b13     datadumpreq001.exp
 0002:00002b50       $N00009                    0000000180007b50     datadumpreq001.exp
 0002:00002b8b       $N00010                    0000000180007b8b     datadumpreq001.exp
 0002:00002bb9       $N00011                    0000000180007bb9     datadumpreq001.exp
 0002:00002bea       $N00012                    0000000180007bea     datadumpreq001.exp
 0002:00002c19       $N00013                    0000000180007c19     datadumpreq001.exp
 0002:00002c48       $N00014                    0000000180007c48     datadumpreq001.exp
 0002:00002c7d       $N00015                    0000000180007c7d     datadumpreq001.exp
 0002:000030e2       .idata$6                   00000001800080e2     kernel32:KERNEL32.dll
 0002:00003146       .idata$6                   0000000180008146     vcruntime:VCRUNTIME140.dll
 0002:000032d8       .idata$6                   00000001800082d8     ucrt:api-ms-win-crt-heap-l1-1-0.dll
 0002:000032f8       .idata$6                   00000001800082f8     ucrt:api-ms-win-crt-runtime-l1-1-0.dll
 0002:0000331a       .idata$6                   000000018000831a     ucrt:api-ms-win-crt-convert-l1-1-0.dll
 0002:0000333c       .idata$6                   000000018000833c     ucrt:api-ms-win-crt-stdio-l1-1-0.dll
 0002:0000335c       .idata$6                   000000018000835c     ucrt:api-ms-win-crt-string-l1-1-0.dll
 0003:00000000       ?codeAttributeName@@3PEBDEB 0000000180009000     libdatadumpreq001.obj
 0003:00000008       ?lineNumberAttributeName@@3PEBDEB 0000000180009008     libdatadumpreq001.obj
 0003:00000010       ?localVarAttributeName@@3PEBDEB 0000000180009010     libdatadumpreq001.obj
 0003:00000018       ?localVarTypeAttributeName@@3PEBDEB 0000000180009018     libdatadumpreq001.obj
 0003:00000020       ?stackMapAttributeName@@3PEBDEB 0000000180009020     libdatadumpreq001.obj
 0003:00000028       ?callBytes@@3PAEA          0000000180009028     libdatadumpreq001.obj
 0003:0000002c       ?allocBytes@@3PAEA         000000018000902c     libdatadumpreq001.obj
 0003:00000030       result                     0000000180009030     libdatadumpreq001.obj
 0003:0001aad4       redefineAttempted          0000000180023ad4     libdatadumpreq001.obj
 0003:0001aad8       nsk_context                0000000180023ad8     libdatadumpreq001.obj
 0003:0001aae4       redefineSucceed            0000000180023ae4     libdatadumpreq001.obj
 0003:0001aae8       agentFailed                0000000180023ae8     libdatadumpreq001.obj
 0003:0001aaec       currentAgentStatus         0000000180023aec     libdatadumpreq001.obj
 0003:0001aaf0       context                    0000000180023af0     libdatadumpreq001.obj
 0003:0001aba8       agentThread                0000000180023ba8     libdatadumpreq001.obj
 0003:0001abb0       agentThreadProc            0000000180023bb0     libdatadumpreq001.obj
 0003:0001abb8       agentThreadArg             0000000180023bb8     libdatadumpreq001.obj
 0003:0001abc0       agent_data                 0000000180023bc0     libdatadumpreq001.obj
 0003:0001abd0       jvmti_env                  0000000180023bd0     libdatadumpreq001.obj
 0003:0001abd8       jvm                        0000000180023bd8     libdatadumpreq001.obj
 0003:0001abe0       jni_env                    0000000180023be0     libdatadumpreq001.obj
 0003:0001abe8       checkStatus_func           0000000180023be8     libdatadumpreq001.obj
 0003:0001abf0       ?codeAttributeIndex@@3GA   0000000180023bf0     libdatadumpreq001.obj
 0003:0001abf2       eventReceived              0000000180023bf2     libdatadumpreq001.obj
 0003:0001abf4       ?lineNumberAttributeIndex@@3GA 0000000180023bf4     libdatadumpreq001.obj
 0003:0001abf8       ?localVarAttributeIndex@@3GA 0000000180023bf8     libdatadumpreq001.obj
 0003:0001abfc       ?localVarTypeAttributeIndex@@3GA 0000000180023bfc     libdatadumpreq001.obj
 0003:0001ac00       ?stackMapAttributeIndex@@3GA 0000000180023c00     libdatadumpreq001.obj
 0003:0001ac04       ?stackFrameOffset@@3GA     0000000180023c04     libdatadumpreq001.obj
 0003:0001ac08       ?mode@@3HA                 0000000180023c08     libdatadumpreq001.obj
 0003:0001ac0c       ?constantPoolSize@@3GA     0000000180023c0c     libdatadumpreq001.obj
 0003:0001ac10       ?orig@@3PEBEEB             0000000180023c10     libdatadumpreq001.obj
 0003:0001ac18       ?gen@@3PEAEEA              0000000180023c18     libdatadumpreq001.obj
 0003:0001ac20       ?inputPos@@3PEAEEA         0000000180023c20     libdatadumpreq001.obj
 0003:0001ac28       ?endPos@@3PEBEEB           0000000180023c28     libdatadumpreq001.obj
 0003:0001ac30       ?genPos@@3PEAEEA           0000000180023c30     libdatadumpreq001.obj
 0003:0001ac38       ?markPos@@3PEAEEA          0000000180023c38     libdatadumpreq001.obj
 0003:0001ac40       ?constantPool@@3PEAPEADEA  0000000180023c40     libdatadumpreq001.obj
 0003:0001ac48       ?constantPoolCount@@3GA    0000000180023c48     libdatadumpreq001.obj
 0003:0001ac4c       ?zeroBytes@@3PAEA          0000000180023c4c     libdatadumpreq001.obj
 0003:0001ac50       ?codeLength@@3IA           0000000180023c50     libdatadumpreq001.obj
 0003:0001ac58       ?map@@3PEAIEA              0000000180023c58     libdatadumpreq001.obj
 0003:0001ac60       ?widening@@3PEACEA         0000000180023c60     libdatadumpreq001.obj
 0003:0001ac68       jvmti                      0000000180023c68     libdatadumpreq001.obj
 0003:0001ac70       callbacks                  0000000180023c70     libdatadumpreq001.obj
 0003:0001ada8       dataDumpRequestMonitor     0000000180023da8     libdatadumpreq001.obj
 0003:0001adc0       GS_ExceptionRecord         0000000180023dc0     MSVCRT:gs_report.obj
 0003:0001ae60       GS_ContextRecord           0000000180023e60     MSVCRT:gs_report.obj
 0003:0001b330       ?g_tss_cv@@3U_RTL_CONDITION_VARIABLE@@A 0000000180024330     MSVCRT:thread_safe_statics.obj
 0003:0001b338       ?g_tss_event@@3PEAXEA      0000000180024338     MSVCRT:thread_safe_statics.obj
 0003:0001b340       ?g_tss_mutex@@3U_RTL_CRITICAL_SECTION@@A 0000000180024340     MSVCRT:thread_safe_statics.obj
 0003:0001b368       ?g_sleep_condition_variable_cs@@3P6AHPEAU_RTL_CONDITION_VARIABLE@@PEAU_RTL_CRITICAL_SECTION@@K@ZEA 0000000180024368     MSVCRT:thread_safe_statics.obj
 0003:0001b370       ?g_wake_all_condition_variable@@3P6AXPEAU_RTL_CONDITION_VARIABLE@@@ZEA 0000000180024370     MSVCRT:thread_safe_statics.obj
 0003:0001b37c       ?__proc_attached@@3HA      000000018002437c     MSVCRT:dll_dllmain.obj
 0003:0001b390       ?is_initialized_as_dll@@3_NA 0000000180024390     MSVCRT:utility.obj
 0003:0001b391       ?module_local_atexit_table_initialized@@3_NA 0000000180024391     MSVCRT:utility.obj
 0003:0001b398       ?module_local_atexit_table@@3U_onexit_table_t@@A 0000000180024398     MSVCRT:utility.obj
 0003:0001b3b0       ?module_local_at_quick_exit_table@@3U_onexit_table_t@@A 00000001800243b0     MSVCRT:utility.obj
